:020000002136A7
:1D000300C000C0E07422253C253CF8C2AF863A08863BD2AFD203D0E0D000C2A832C4
:020023002103B7
:20002B00C2CFC0E0C0F0C082C083C0D0752100E522700FE523700B7C00A2B79286B3928767
:20004B000199D208E52615267044E514C39CFB50027B00E5237007E514C395225001E4F5EB
:20006B00F0C39BEB4002E5F08510F0A42528F526E522700215231522BCFF027CFE0CE52A5A
:20008B00252CF52C540F252E90032693F580E524700FE525700B7D00A2B792A6B392A70164
:2000AB00F8D209E52715277044E515C39DFB50027B00E5257007E515C395245001E4F5F033
:2000CB00C39BEB4002E5F08511F0A42529F527E524700215251524BDFF027DFE0DE52B25B8
:2000EB002DF52D540F252F90032693F5A0D0D0D083D082D0F0D0E03230982FC0E0C0D0C23E
:20010B0098A79930000AB74207200216D2028939300207B70D04C202D20109430180EAB5F0
:20012B000104D2B380FED0D0D0E032758E0175813D758780758922E5B0C4540790031E935F
:20014B00F58DF58BD288D28E759852783C760018B801FAD2007A8079807402F510F51174CA
:20016B0032F512F51375CBFF75CA4775C80475A8B075B820C2B3318F31AF51E980F8318F8C
:20018B003000FB22EAB50101223099FDC2998A008699C200B60D02D2000A4302802285F0BB
:2001AB0039C20122200101220539433980A839E6C3943040E9F538940950E37531078539B9
:2001CB00F00539433980A839E6C3943040D0940A50CCD531EC85F039753707053943398045
:2001EB00A839E6C39430C0E0E537242FF8D0E0F6D537E8E53375F00AA42532F532E53575CD
:20020B00F00AA4253475F064A42532F532E435F0F533E53175F00AA42530F530E536F534D9
:20022B005406232323F535E536540175360160037536FFE538B40021E512C395285001E4FF
:20024B008510F084C2CA85322285332385302885352E85362AF51441C4B40121E513C3956C
:20026B00295001E48511F084C2CA85322485332585302985352F85362BF51541C4B404054E
:20028B0085329041C4B4050451DA41C4B4060985343CC289D2A841C4B40717533401E53425
:2002AB002410F8E5306016A630E5342412F8A63241C4B4080851CB41C4D2CAB2B3C20122B7
:2002CB00318974427116E521710B740D711622318974427116E5907101740D711622300335
:2002EB0014318974427116E53B7101E53A7101740D7116C20322C0E0C4710BD0E0710B22A8
:20030B00540FB40A004002240724303099FDC299F59922FFFEFDFAF4E8D0A0606444406037
:20032B00644440606444406064444043495869636D5C4D43495869636D5C4D434249505838
:1B034B0070696263666D745C544D46434249505870696263666D745C544D46D1
:00000001FF
